:100000000C942B060C941F080C942A080C94480698
:100010000C94C90F0C9448060C9448060C9448069E
:100020000C9448060C9448060C9448060C94480618
:100030000C9448060C9448060C9448060C94480608
:100040000C9448060C9448060C9435080C94480609
:100050000C9448062020202052616E646F6D00547D
:10006000524700444953004F4646004F4E200090EF
:100070000200004B064809580966069D060E090E47
:10008000097F020000D40648095809EB06F3060E62
:10009000090E09E6010000FC06480958090F071B74
:1000A000070E090E09D5010000270748095809471E
:1000B00007500713091309C40100005F07480958D6
:1000C000098907CB070E090E09B3010000440C484B
:1000D000095809600C970CBE110E09F602130AF6B6
:1000E0000CE508F908020D380D99113F09E50213D6
:1000F00009F60CE508F908020D380D99113F09D4ED
:10010000021306F60CE508F908020D380D99113FA7
:1001100009C3021308F60CE508F908020D380D9919
:10012000113F09B2021307F60CE508F908020D3871
:100130000D99113F09A1021305F60CE508F9080213
:100140000D380D99113F096E0200007F09E508F98D
:10015000084A064A06160E3F095D0200008B09E5B3
:1001600008F908E6095C0AEA113F094C0200007B25
:100170000EE508F9080E101910A5123F093B020000
:1001800000BD0EC10ED00E020D380DB1113F092A6F
:10019000020000DF0E280F3C0F500F740FCC123FEF
:1001A0000919020000D20AF5080A092A0BC10BE15D
:1001B000133F092043616C69627261746520467265
:1001C0006571200020547269676765722044656C10
:1001D0006179202000202053796E63204F75747060
:1001E0007574202020002020204F6666204C657604
:1001F000656C20202020002020202020537765657A
:1002000070202053746570002020202020537765D3
:100210006570202020456E64002020202020537728
:10022000656570202020202020002050574D202878
:10023000485329202020202020200020202020207A
:100240002050574D20202020202020002020204812
:100250006967682053706565642020200020202095
:10026000202050756C736520202020202000202045
:100270002020204E6F697365202020202020002040
:10028000202046726571204D6F646520202020007B
:100290002020204672657120537465702020202034
:1002A00000202020202020454347202020202020FF
:1002B0002000202052657620536177546F6F746858
:1002C00020200020202020536177546F6F74682015
:1002D0002020200020202020547269616E676C6508
:1002E000202020200020202020205371756172657D
:1002F00020202020200020202020202053696E650F
:1003000020202020202000130A13091306130813AD
:100310000713050A0E2D73C440AA8FDDF36B97B93E
:100320008D7757E352933F2507995F8B37307B3AA0
:1003300089C6AE4E58E44B4805D6F25C44EFF869E6
:10034000F692561D96AB2F8835F53683FC8E60E00D
:10035000DAA85BDF7E4D3B38912BFA21C2230D2EAC
:10036000CE3CB60332ED86E60F556A34B870454987
:100370009B76BC185A414628FD2CB0EAB2DE65BB1C
:100380001059F19DB729D4EB42856F39D526907F5E
:10039000A7E8D998C18C1162AD81660C5D19011E68
:1003A000C887E12AD224D143E74F68C0AF5E9E845C
:1003B000E250CB1AC3B47404AC64A013D331009CD4
:1003C000FE4AB378153EEE947C1C72A1209F95CF17
:1003D0003D82B5BD54A6476E75C71BD70916F012EE
:1003E00002B1064CCDA9A26CA561CA7D1F221714CB
:1003F000C5D86D8AF751A3FBF463BF79C927EC7A9E
:100400009ABE80FFE5BACC0BDBDCF967E9A408D023
:1004100071335300000000000000000000000101E3
:100420000203030405060708090A0C0D0F10121336
:100430001517191B1D1F212325272A2C2E31333672
:10044000383B3E404346494C4F5154575A5D6063D8
:10045000676A6D707376797C808386898C8F9295BC
:10046000989C9FA2A5A8ABAEB0B3B6B9BCBFC1C49F
:10047000C7C9CCCED1D3D5D8DADCDEE0E2E4E6E8F9
:10048000EAECEDEFF0F2F3F5F6F7F8F9FAFBFCFC25
:10049000FDFEFEFFFFFFFFFFFFFFFFFFFFFFFEFE72
:1004A000FDFCFCFBFAF9F8F7F6F5F3F2F0EFEDECF2
:1004B000EAE8E6E4E2E0DEDCDAD8D5D3D1CECCC996
:1004C000C7C4C1BFBCB9B6B3B0AEABA8A5A29F9C10
:1004D0009895928F8C898683807C797673706D6A0B
:1004E0006763605D5A5754514F4C494643403E3B09
:1004F000383633312E2C2A272523211F1D1B19178F
:10050000151312100F0D0C0A090807060504030342
:10051000020101494A4B4B4A494949494847454428
:10052000434343444443413E3D3B393837373636F5
:1005300036373737373737363533323131343D4D4B
:100540006584A9CFEEFFFEEAC69A6D442511050029
:1005500001060D141C242D34393D404142434444CE
:100560004546474747474747474748484849494A14
:100570004B4B4C4D4E4F505152535456585B5D604F
:10058000626466686B6D707376797B7D7E7F7F7F3A
:100590007F7F7E7D7C797774716D6966625F5C595F
:1005A0005754514F4D4C4B4A4948464544434343A9
:1005B0004444444545454545454546474849494ADB
:1005C0004A4B4B4B4B4B4B4A4A494949494848488F
:1005D00047474747474747464646454545454546B9
:1005E00046464544444343434342424241414141DC
:1005F0004141414140403F3F4040414141414141F3
:1006000041404040404040404041414142434445D8
:1006100047484900020406080A0C0E101214161866
:100620001A1C1E20222426282A2C2E30323436383A
:100630003A3C3E40424446484A4C4E50525456582A
:100640005A5C5E60626466686A6C6E70727476781A
:100650007A7C7E80828486888A8C8E90929496980A
:100660009A9C9EA0A2A4A6A8AAACAEB0B2B4B6B8FA
:10067000BABCBEC0C2C4C6C8CACCCED0D2D4D6D8EA
:10068000DADCDEE0E2E4E6E8EAECEEF0F2F4F6F8DA
:10069000FAFCFEFFFDFBF9F7F5F3F1EFEFEBE9E70D
:1006A000E5E3E1DFDDDBD9D7D5D3D1CFCFCBC9C7E8
:1006B000C5C3C1BFBDBBB9B7B5B3B1AFAFABA9A7D8
:1006C000A5A3A19F9D9B99979593918F8F8B8987C8
:1006D0008583817F7D7B79777573716F6F6B6967B8
:1006E0006563615F5D5B59575553514F4F4B4947A8
:1006F0004543413F3D3B39373533312F2F2B292798
:100700002523211F1D1B19171513110F0F0B090787
:10071000050301FFFEFDFCFBFAF9F8F7F6F5F4F32B
:10072000F2F1F0EFEEEDECEBEAE9E8E7E6E5E4E321
:10073000E2E1E0DFDEDDDCDBDAD9D8D7D6D5D4D311
:10074000D2D1D0CFCECDCCCBCAC9C8C7C6C5C4C301
:10075000C2C1C0BFBEBDBCBBBAB9B8B7B6B5B4B3F1
:10076000B2B1B0AFAEADACABAAA9A8A7A6A5A4A3E1
:10077000A2A1A09F9E9D9C9B9A99989796959493D1
:100780009291908F8E8D8C8B8A89888786858483C1
:100790008281807F7E7D7C7B7A79787776757473B1
:1007A0007271706F6E6D6C6B6A69686766656463A1
:1007B0006261605F5E5D5C5B5A5958575655545391
:1007C0005251504F4E4D4C4B4A4948474645444381
:1007D0004241403F3E3D3C3B3A3938373635343371
:1007E0003231302F2E2D2C2B2A2928272625242361
:1007F0002221201F1E1D1C1B1A1918171615141351
:100800001211100F0E0D0C0B0A0908070605040340
:10081000020100000102030405060708090A0B0C87
:100820000D0E0F101112131415161718191A1B1C80
:100830001D1E1F202122232425262728292A2B2C70
:100840002D2E2F303132333435363738393A3B3C60
:100850003D3E3F404142434445464748494A4B4C50
:100860004D4E4F505152535455565758595A5B5C40
:100870005D5E5F606162636465666768696A6B6C30
:100880006D6E6F707172737475767778797A7B7C20
:100890007D7E7F808182838485868788898A8B8C10
:1008A0008D8E8F909192939495969798999A9B9C00
:1008B0009D9E9FA0A1A2A3A4A5A6A7A8A9AAABACF0
:1008C000ADAEAFB0B1B2B3B4B5B6B7B8B9BABBBCE0
:1008D000BDBEBFC0C1C2C3C4C5C6C7C8C9CACBCCD0
:1008E000CDCECFD0D1D2D3D4D5D6D7D8D9DADBDCC0
:1008F000DDDEDFE0E1E2E3E4E5E6E7E8E9EAEBECB0
:10090000EDEEEFF0F1F2F3F4F5F6F7F8F9FAFBFC9F
:10091000FDFEFF00000000000000000000000000DD
:1009200000000000000000000000000000000000C7
:1009300000000000000000000000000000000000B7
:1009400000000000000000000000000000000000A7
:100950000000000000000000000000000000000097
:100960000000000000000000000000000000000087
:100970000000000000000000000000000000000077
:100980000000000000000000000000000000000067
:10099000000000FFFFFFFFFFFFFFFFFFFFFFFFFF64
:1009A000FFFFFFFFFFFFFFFFFFFFFFFFFFFFFFFF57
:1009B000FFFFFFFFFFFFFFFFFFFFFFFFFFFFFFFF47
:1009C000FFFFFFFFFFFFFFFFFFFFFFFFFFFFFFFF37
:1009D000FFFFFFFFFFFFFFFFFFFFFFFFFFFFFFFF27
:1009E000FFFFFFFFFFFFFFFFFFFFFFFFFFFFFFFF17
:1009F000FFFFFFFFFFFFFFFFFFFFFFFFFFFFFFFF07
:100A0000FFFFFFFFFFFFFFFFFFFFFFFFFFFFFFFFF6
:100A1000FFFFFF808386898C8F9295989C9FA2A56B
:100A2000A8ABAEB0B3B6B9BCBFC1C4C7C9CCCED1F8
:100A3000D3D5D8DADCDEE0E2E4E6E8EAECEDEFF08C
:100A4000F2F3F5F6F7F8F9FAFBFCFCFDFEFEFFFF0A
:100A5000FFFFFFFFFFFFFFFFFFFEFEFDFCFCFBFAB9
:100A6000F9F8F7F6F5F3F2F0EFEDECEAE8E6E4E298
:100A7000E0DEDCDAD8D5D3D1CECCC9C7C4C1BFBC87
:100A8000B9B6B3B0AEABA8A5A29F9C9895928F8C37
:100A9000898683807C797673706D6A6763605D5A3E
:100AA0005754514F4C494643403E3B383633312E24
:100AB0002C2A272523211F1D1B1917151312100F70
:100AC0000D0C0A09080706050403030201010000D2
:100AD0000000000000000000000101020303040503
:100AE000060708090A0C0D0F1012131517191B1D04
:100AF0001F212325272A2C2E313336383B3E4043F5
:100B000046494C4F5154575A5D6063676A6D707324
:100B100076797C001F000000001F00001F101010DD
:100B2000101F00001F181818181F00001F1C1C1C85
:100B30001C1F00001F1E1E1E1E1F00001F1F1F1F48
:100B40001F1F0003070F1F0F070300181C1E1F1E87
:100B50001C18006E616E00696E660000407A10F32A
:100B60005A00A0724E18090010A5D4E80000E876DB
:100B700048170000E40B54020000CA9A3B00000032
:100B8000E1F505000080969800000040420F00004B
:100B900000A08601000000102700000000E803000C
:100BA0000000006400000000000A000000000001D6
:100BB00000000000002C76D888DC674F0823DFC1D6
:100BC000DFAE59E1B1B796E5E3E453C63AE6519991
:100BD0007696E8E6C28426EB898C9B62ED407C6FBA
:100BE000FCEFBC9C9F40F2BAA56FA5F490055A2A71
:100BF000F75C936B6CF9676DC11BFCE0E40D47FE7D
:100C0000F520E6B500D0ED902E0300943577050071
:100C100080841E080000204E0A000000C80C3333F8
:100C200033330F986E12831141EF8D2114893BE607
:100C30005516CFFEE6DB18D1844B381BF77C1D9090
:100C40001DA4BBE424203284725E228100C9F124F9
:100C5000ECA1E53D270011241FBECFE5D4E0DEBFA7
:100C6000CDBF11E0A0E6B0E0E2EEFBE302C00590EC
:100C70000D92AE32B107D9F711E0AEE2B1E001C09A
:100C80001D92A335B107E1F70E94BA150C94EF1D30
:100C90000C940000089561E080E00E948B14E3E76B
:100CA000F0E083818F9382818F9381818F93808104
:100CB0008F9383E990E09F938F930E94371D0F904D
:100CC0000F900F900F900F900F900895CF92DF929A
:100CD000EF92FF9220E030E040E251E46091730037
:100CE0007091740080917500909176000E94A31914
:100CF0006B017C012FE632E143E85AE30E949F1921
:100D000087FD09C0C0927300D0927400E092750014
:100D1000F09276000CC08FE692E1A3E8BAE38093EC
:100D2000730090937400A0937500B0937600FF90C9
:100D3000EF90DF90CF900C944B06CF92DF92EF9222
:100D4000FF9220E030E040E251E460917300709146
:100D5000740080917500909176000E94ED1A6B01ED
:100D60007C0120E030E44CE156E40E94E91A1816B8
:100D70004CF0C0927300D0927400E0927500F09233
:100D800076000CC080E090E4ACE1B6E480937300A0
:100D900090937400A0937500B0937600FF90EF904D
:100DA000DF90CF900C944B0661E080E00E948B14A2
:100DB00080917700882319F0813021F008958CE923
:100DC00090E002C088EA90E09F938F930E94371DC5
:100DD0000F900F90089580917700813011F4109258
:100DE00077000C94D40680917700811103C081E0D4
:100DF000809377000C94D40661E080E00E948B140D
:100E000080917B001F928F9384EB90E09F938F9350
:100E10000E94371D0F900F900F900F9008958091B2
:100E20007B00882319F0815080937B0080917B00A8
:100E30008BBB0C94FC0680917B008F3F19F08F5F79
:100E400080937B0080917B008BBB0C94FC0661E05F
:100E500080E00E948B1480918000813049F028F05E
:100E6000823049F0833051F0089588EB90E008C05B
:100E700081EC90E005C08AEC90E002C083ED90E048
:100E80009F938F930E94371D0F900F90089580912C
:100E90008000882319F08150809380000C942707EC
:100EA000809180008F5F843009F483E0809380001C
:100EB0000C9427070E94181480E090E0089561E0E8
:100EC00080E00E948B14809180008330C9F480916F
:100ED00084008F93809183008F93809182008F9301
:100EE000809181008F938CED90E09F938F930E946F
:100EF000371D0F900F900F900F900F900F90089547
:100F000084EE90E09F938F930E94371D0F900F9077
:100F10000895CF92DF92EF92FF9283E0809380005A
:100F200020E030E048EC52E460917300709174006E
:100F300080917500909176000E94A3199B01AC01ED
:100F40006091810070918200809183009091840073
:100F50000E943A196B017C012FE632E143E85AE323
:100F60000E949F1987FD09C0C0928100D092820023
:100F7000E0928300F092840008C0109281001092E9
:100F800082001092830010928400FF90EF90DF9017
:100F9000CF900C945F07CF92DF92EF92FF9283E0A5
:100FA0008093800020E030E048EC52E460917300D0
:100FB0007091740080917500909176000E94A31941
:100FC00020918100309182004091830050918400F3
:100FD0000E943B196B017C0120E030E04AE754E4B9
:100FE0000E94E91A18164CF0C0928100D09282003B
:100FF000E0928300F09284000CC080E090E0AAE7C9
:10100000B4E48093810090938200A0938300B09316
:101010008400FF90EF90DF90CF900C945F0714BC9A
:10102000089585B5866085BD89B7806489BF0895B8
:1010300083B7897F83BF89B78F7B89BF08951F924C
:101040000F920FB60F9211246A9A0F900FBE0F9055
:101050001F9018951F920F920FB60F9211246A9A43
:101060000F900FBE0F901F9018951F920F920FB602
:101070000F9211246A9A0F900FBE0F901F9018952F
:1010800080912F01909130010196909330018093CF
:101090002F01849B0CC0839B0CC0809B0CC0819B48
:1010A0000CC0829B0CC086990CC046E00BC041E08E
:1010B00009C042E007C043E005C044E003C045E08A
:1010C00001C040E020913601241769F041112EC083
:1010D0002091310130913201BC01621B730B6431EC
:1010E000710590F123C020913601222369F14091CE
:1010F00035012091310130913201411107C0AC011D
:10110000421B530B4436510538F40895BC01621B51
:10111000730B68307105C0F0109237019093340161
:101120008093330181E080933501089590933201DB
:10113000809331014093360110923701909334012E
:101140008093330110923501089544E250E060E04D
:1011500070E081E690E00C94C11D8FEF91E00E9459
:10116000B91D843539F00E94A50864E58FEF91E040
:101170000E94E21D44E250E060E070E081E690E011
:101180000C94A91D6091610082E1689FB001112457
:1011900065527F4F42E150E089E391E00E94E61CF6
:1011A0008FE391E090934C0180934B010E94661471
:1011B00040E060E08091390190913A010E949914D9
:1011C000E0913D01F0913E01099480913801811137
:1011D0000BC080916100811102C08BE001C0815081
:1011E000809361000C94C208089510922E010C9413
:1011F000E5088091380181110CC0809161008F5FFA
:101200008C3019F08093610002C0109261000C9440
:10121000C208089510922E010C94F9088FEF809364
:1012200060000C94C20880918000833011F08D9A88
:1012300001C08D980C940E096091600082E1689F56
:10124000B001112461597F4F42E150E089E391E000
:101250000E94E61C8FE391E090934C0180934B0138
:101260000E94661440E060E08091390190913A015B
:101270000E949914E0913D01F0913E010994809102
:101280003801811104C0109260000C941C0908956B
:101290008091380181110BC080916000811102C0E2
:1012A00085E001C08150809360000C941C09089572
:1012B0008091380181110CC0809160008F5F863071
:1012C00019F08093600002C0109260000C941C0919
:1012D000089580913801882361F0809180008330E7
:1012E00019F48FE590E002C08BE690E041E06DE0FC
:1012F00004C041E06DE087E690E00C94991461E051
:1013000080E00E948B1441E060E084E590E00E9460
:1013100099140C9469090F931F93CF93DF9361E0A5
:1013200080E00E948B14C0917C00D0917D001091D0
:101330007E0000917F002FEF3FEF4FE75FEFF80156
:101340006C2F7D2F8F2F9E2F0E949F1987FF03C028
:101350008FEE90E00EC020E030E0A901F8016C2F84
:101360007D2F8F2F9E2F0E949F19811109C08AEF18
:1013700090E09F938F930E94371D0F900F9020C095
:101380002FEF3FEF4FE75FE7F8016C2F7D2F8F2F97
:101390009E2F0E94E91A18161CF485E091E0E9CF0F
:1013A0000F931F93DF93CF938CED90E09F938F93D8
:1013B0000E94371D0F900F900F900F900F900F907D
:1013C000DF91CF911F910F910C946909CF92DF9219
:1013D000EF92FF9280913801811169C0C0907C002A
:1013E000D0907D00E0907E00F0907F002FEF3FEFE7
:1013F0004FE75FEFC701B6010E949F1987FD51C0FB
:1014000020E030E0A901C701B6010E949F198111B7
:1014100005C080E090E0A0E8BFEF0EC02FEF3FEFE7
:101420004FE75FE7C701B6010E94E91A18166CF48E
:1014300080E090E0AAE7B4E480937C0090937D0084
:10144000A0937E00B0937F002CC020E030E048ECF9
:1014500052E46091730070917400809175009091D6
:1014600076000E94A3199B01AC01C701B6010E943E
:101470003A1960937C0070937D0080937E00909376
:101480007F002FE632E143E85AE30E949F1987FF6D
:1014900008C010927C0010927D0010927E00109285
:1014A0007F00FF90EF90DF90CF900C948B09FF901E
:1014B000EF90DF90CF900895CF92DF92EF92FF925E
:1014C00080913801811169C0C0907C00D0907D006E
:1014D000E0907E00F0907F002FEF3FEF4FE75FEF4F
:1014E000C701B6010E949F1987FF09C010927C00B6
:1014F00010927D0010927E0010927F0048C020E084
:1015000030E0A901C701B6010E949F19811105C0F1
:101510008FE692E1A3E8BAE332C02FEF3FEF4FE747
:101520005FE7C701B6010E94E91A181684F120E0AE
:1015300030E048EC52E46091730070917400809147
:101540007500909176000E94A3199B01AC01C70120
:10155000B6010E943B1960937C0070937D008093DC
:101560007E0090937F0020E030E04AE754E40E9440
:10157000E91A181664F480E090E0A0E8BFE78093D1
:101580007C0090937D00A0937E00B0937F00FF903D
:10159000EF90DF90CF900C948B09FF90EF90DF904D
:1015A000CF90089580912E01813081F1C8F0823072
:1015B00009F04EC040E060E087EF91E00E9499148E
:1015C00061E080E00E948B14809171008F93809184
:1015D00070008F9380916F008F9380916E002BC06D
:1015E00040E060E089E192E00E94991461E080E0CF
:1015F0000E948B14809165008F93809164008F937B
:10160000809163008F938091620015C040E060E09C
:1016100088E092E00E94991461E080E00E948B14BF
:1016200080916D008F9380916C008F9380916B00FF
:101630008F9380916A008F9383E990E09F938F93BB
:101640000E94371D0F900F900F900F900F900F90EA
:101650000C946909CF92DF92EF92FF9280912E0154
:10166000813079F120F0823009F45CC084C020918F
:101670007300309174004091750050917600609134
:1016800062007091630080916400909165000E94F7
:101690003A196093620070936300809364009093A2
:1016A000650020E030E0A9010E949F1987FF63C018
:1016B0001092620010926300109264001092650014
:1016C0005AC0209173003091740040917500509180
:1016D000760060916A0070916B0080916C0090912F
:1016E0006D000E943A1960936A0070936B008093BA
:1016F0006C0090936D00C0906200D0906300E09009
:101700006400F0906500A70196010E949F1987FF71
:1017100032C0C0926A00D0926B00E0926C00F092EE
:101720006D0029C0209173003091740040917500C4
:101730005091760060916E0070916F008091700002
:10174000909171000E943A1960936E0070936F003F
:10175000809370009093710020E030E0A9010E9416
:101760009F1987FF08C010926E0010926F001092B0
:10177000700010927100FF90EF90DF90CF900C946A
:10178000D20A80912E01813001F120F0823009F4DB
:101790004BC078C020917300309174004091750067
:1017A00050917600609162007091630080916400B6
:1017B000909165000E943B196093620070936300F2
:1017C00080936400909365001AC02091730030915B
:1017D0007400409175005091760060916A0070919C
:1017E0006B0080916C0090916D000E943B1960939A
:1017F0006A0070936B0080936C0090936D0020E002
:1018000034E244E758E40E94E91A1816DCF580E057
:1018100094E2A4E7B8E48093620090936300A093FD
:101820006400B09365002EC0209173003091740065
:10183000409175005091760060916E0070916F003C
:1018400080917000909171000E943B1960936E002E
:1018500070936F00809370009093710020E030E0EF
:1018600048EC52E40E94E91A181664F480E090E013
:10187000A8ECB2E480936E0090936F00A093700088
:10188000B09371000C94D20A61E080E00E948B1446
:10189000E6E6F0E083818F9382818F9381818F933D
:1018A00080818F9380E191E09F938F930E94371DF9
:1018B0000F900F900F900F900F900F900C9469095C
:1018C000CF92DF92EF92FF922DEB37E346E855E39C
:1018D0006091660070916700809168009091690046
:1018E0000E943A196B017C012CEE31E548EB5DE377
:1018F0000E949F1987FD09C0C0926600D0926700C0
:10190000E0926800F09269000CC08CEE91E5A8EBC3
:10191000BDE38093660090936700A0936800B09346
:101920006900FF90EF90DF90CF900C94440CCF9221
:10193000DF92EF92FF922DEB37E346E855E360919B
:1019400066007091670080916800909169000E9424
:101950003B196B017C012EEA37E441E85FE30E940A
:10196000E91A18164CF0C0926600D0926700E09217
:101970006800F09269000CC08EEA97E4A1E8BFE32A
:101980008093660090936700A0936800B09369000D
:10199000FF90EF90DF90CF900C94440C0F931F9327
:1019A000CF93DF9300D0CDB7DEB7162F082F61E0BD
:1019B00080E079839A830E948B149A819F930F937E
:1019C00079817F931F9383E990E09F938F930E9487
:1019D000371D0F900F900F900F900F900F900F905A
:1019E0000F90DF91CF911F910F9108956091620048
:1019F0007091630080916400909165000E94CE0C0C
:101A00000C946909CF92DF92EF92FF9220917300BC
:101A100030917400409175005091760060916200A1
:101A20007091630080916400909165000E943A1962
:101A30006B017C0120E030E0A9010E949F1987FD25
:101A400009C0C0926200D0926300E0926400F092FC
:101A5000650008C01092620010926300109264004A
:101A600010926500FF90EF90DF90CF900C94F60CF1
:101A7000CF92DF92EF92FF92209173003091740029
:101A80004091750050917600609162007091630002
:101A900080916400909165000E943B196B017C016C
:101AA00020E034E244E758E40E94E91A18164CF0AA
:101AB000C0926200D0926300E0926400F0926500F0
:101AC0000CC080E094E2A4E7B8E4809362009093B5
:101AD0006300A0936400B0936500FF90EF90DF90E7
:101AE000CF900C94F60C809136018111FCCF8BB70E
:101AF000806E8BBF0C9418088BB78F718BBF0C94C2
:101B000011080E94A50881E080933801E0913D0111
:101B1000F0913E0109950C94730DCF92DF92EF92F4
:101B2000FF926B017C01642F70E080E090E00E94E6
:101B3000391A9B01AC0160E074E284E79BE40E94E7
:101B4000A31920E030E040E853E30E94ED1A20E0C2
:101B500030E040E85BE30E94ED1A2091660030918E
:101B6000670040916800509169000E94A3199B0191
:101B7000AC01C701B6010E94A3190E940B1AFF9085
:101B8000EF90DF90CF900895CF92DF92EF92FF9287
:101B9000CF93DF931F92CDB7DEB749830E94371AE8
:101BA0006B017C014981642F70E080E090E00E942D
:101BB000391A9B01AC0160E074E284E79BE40E9467
:101BC000A31920E030E040E853E30E94ED1A20E042
:101BD00030E040E85BE30E94ED1A2091660030910E
:101BE000670040916800509169000E94A3199B0111
:101BF000AC01C701B6010E94ED1A0F90DF91CF91A1
:101C0000FF90EF90DF90CF9008950E947C0D10928E
:101C1000380180917B008BBBE0913D01F0913E014A
:101C20000995809136018111FCCF08950E94810DA4
:101C30006A9840E051E063E173E080E092E00E9446
:101C4000E61C809180009FEF980F923010F4959AD7
:101C50009598833059F58D986A9820E030E04AE7EE
:101C600056E4609181007091820080918300909190
:101C700084000E94ED1A20E030E040EC50E40E9425
:101C8000A3190E940B1A611571058105910539F49C
:101C900085990CC06A9BFCCF16C06A9914C0859BBD
:101CA000FCCF6150704080409040D9F7E0E0F2E016
:101CB0002CEF322F00800BBAE3953A9511F4322FB6
:101CC000E02D6A9BF7CF0C94050E80918000833045
:101CD00061F080913801882319F08BE690E002C012
:101CE00087E690E041E06DE004C041E06DE083E60E
:101CF00090E00C94991461E080E00E948B14809134
:101D000072001F928F9386E191E09F938F930E94C0
:101D1000371D0F900F900F900F900C94650E60E0A0
:101D20008AE00E948B1460917A0070E080E090E07D
:101D30000E94371A20E030E040E85FE30E943B1940
:101D400020E030E040E85BE30E94ED1A20E030E064
:101D500048EC52E40E94ED1A9F938F937F936F9308
:101D60008EE191E09F938F930E94371D0F900F900B
:101D70000F900F900F900F9008950E94F60C0C9406
:101D80008F0E80913801811102C00C94E50880917A
:101D90007A008F3F19F08F5F80937A000C94BD0E0C
:101DA00080913801811102C00C94F90880917A0069
:101DB000882319F0815080937A000C94BD0E0F9304
:101DC0001F93CF93DF938091780090917900843FA7
:101DD0009105F1F038F4CD97B1F4C6EFD8E214E7ED
:101DE00002E41AC0803D23E0920741F085389E410D
:101DF00051F4C0E0D4E214EF05E40EC0C7EDD3E225
:101E000014E704E409C0C0E0D4E214E707E404C026
:101E1000C7EDD3E214E703E40E948F0E61E080E097
:101E20000E948B140F931F93DF93CF9386E291E070
:101E30009F938F930E94371D0F900F900F900F90DC
:101E40000F900F90DF91CF911F910F910C94650E21
:101E500080913801811102C00C94E50880917A00CC
:101E60008F3F19F08F5F80937A0080917A0090E025
:101E70009BBD8ABD0C94DF0E80913801811102C098
:101E80000C94F90880917A00882319F0815080938E
:101E90007A0080917A0090E09BBD8ABD0C94DF0EA1
:101EA0008091780090917900803D23E0920789F03D
:101EB00030F4843F9105B1F48DE390E00FC0853894
:101EC0002EE1920749F08432944F61F485E89EE157
:101ED00005C084EF90E002C080ED93E0909379001C
:101EE000809378000C94DF0E8091780090917900B7
:101EF000843F910581F028F4CD97B1F484EF90E010
:101F00000FC0803D23E0920749F085389E4161F47F
:101F100084E294EF05C080ED93E002C085E89EE185
:101F200090937900809378000C94DF0E20917A00D2
:101F300080E0E82FF0E0E050FE4F91E0281708F431
:101F400090E0919590838F3F11F08F5FF2CF0895CD
:101F5000CF92DF92EF92FF926B017C01209166009D
:101F60003091670040916800509169006EE873E01D
:101F700089ED9DE30E94A3199B01AC01C701B60145
:101F80000E94A3190E940B1AFF90EF90DF90CF9050
:101F900008951F920F920FB60F9211242F933F9323
:101FA0004F935F936F937F938F939F93AF93BF9361
:101FB000EF93FF930E944008FF91EF91BF91AF9183
:101FC0009F918F917F916F915F914F913F912F9151
:101FD0000F900FBE0F901F901895843039F0883005
:101FE00041F0823049F483E090E008C081E090E065
:101FF00005C01BBC1ABC04C087E090E09BBD8ABD35
:1020000080E48FBD89E08EBD0895809138018823DA
:1020100021F0809172000C94ED0F08958091720070
:10202000813019F08695809372000E947B0E0C948B
:10203000051080917200883019F0880F809372002B
:102040000E947B0E0C940510843F910591F020F4C2
:10205000CD9769F485E00EC0803D23E0920729F01A
:1020600085389E4121F482E005C083E003C081E011
:1020700001C084E091E89FBD88608EBD08951FBCBB
:102080001EBC089585E890E09093500180934F0125
:102090000E94D6140E9466140E9450150E94AD083A
:1020A0001092380180917B008BBB8FEF8ABB81B38C
:1020B000807A81BB82B38F6582BBBA9884E088BB8B
:1020C00080918000833011F08D9A01C08D9814BCEE
:1020D0000E947C0D0E94C208789408958091370177
:1020E000811143C08091360191E090933701833094
:1020F000E1F028F4813049F0823079F0089585309C
:1021000021F1D8F0863049F10895E0914B01F0912A
:102110004C010190F081E02D27C0E0914B01F0913E
:102120004C010680F781E02D1FC0E0914B01F0913A
:102130004C010280F381E02D17C0E0914B01F0913A
:102140004C010480F581E02D0FC0E0914B01F0912E
:102150004C010084F185E02D07C0E0914B01F09126
:102160004C010284F385E02D099408950E947C0DB2
:1021700080913601882319F00E946E10F9CF0C94DB
:10218000730D9F92AF92BF92CF92DF92EF92FF9228
:102190000F931F93CF93DF93C82F809180008230DD
:1021A00019F42FE0922E02C09AE0992E60916200FD
:1021B000709163008091640090916500492D0E94A8
:1021C0008D0D6B017C01611571058105910521F46F
:1021D000C12CD12C7601C394CC2379F18091770066
:1021E000813059F5D701C60156016D01E12CF12C62
:1021F00000E010E020E030E040E050E061E070E01E
:1022000080E090E00E947A1B59016A017B018C01F9
:1022100020E030E040E050E061E070E080E090E0FD
:102220000E947A1BC22ED32EE42EF52E492DC70113
:10223000B6010E94C40D0E94CE0C6A988091800065
:10224000813039F008F445C0823031F08330B1F08C
:102250004DC0959A95983DC0E0E0F2E01127222705
:1022600033271C0D2D1D3E1DEF1D00800BBAE7FD11
:102270009598E7FF959A6A9BF4CF38C08D986A9835
:1022800020E030E04AE756E46091810070918200DE
:1022900080918300909184000E94ED1A20E030E04C
:1022A00040EC50E40E94A3190E940B1A61157105BD
:1022B0008105910539F485990CC06A9BFCCF16C045
:1022C0006A9914C0859BFCCF61507040804090405B
:1022D000D9F7E0E0F2E01127222733271C0D2D1D4E
:1022E0003E1DEF1D00800BBA6A9BF8CF80917B00EA
:1022F0008BBBDF91CF911F910F91FF90EF90DF90FB
:10230000CF90BF90AF909F900C94B61060913B011E
:1023100070913C0140E051E080E092E00E94E61CB8
:1023200080913801882321F081E00E94C110F8CF0C
:10233000089580913801811106C00E94810D0E948C
:1023400086110C94050E1092380108958091380181
:10235000882331F00E94960F81E00E94C110F6CFD1
:10236000089580913801811106C00E94810D0E945C
:10237000A6110C94050E1092380108958091380131
:10238000811125C081E0809338010E94440C0E9495
:10239000730D40E051E063E174E080E092E00E9460
:1023A000E61C80913801882321F080E00E94C11052
:1023B000F8CF0E947C0D1092380180917B008BBB7E
:1023C0000E94440C809136018111FCCF0895109237
:1023D00038010895CF92DF92EF92FF92CF93DF936F
:1023E00080913801811147C081E0809338010E94BB
:1023F0008B09C1E080918000833009F045C0C0E0C6
:102400008D986A9820E030E04AE756E460918100B8
:102410007091820080918300909184000E94ED1A57
:1024200020E030E040EC50E40E94A3190E940B1A17
:10243000611571058105910539F4859925C06A9B5F
:10244000FCCF0FC06A990DC0859BFCCF61507040D6
:1024500080409040D9F718C0C111959880917B00B9
:102460008BBB10923801DF91CF91FF90EF90DF90FE
:10247000CF900C948B0910923801DF91CF91FF908F
:10248000EF90DF90CF900895C0907C00D0907D00B9
:10249000E0907E00F0907F002FEF3FEF4FE75FEF7F
:1024A000C701B6010E949F1987FF0BC0C111959A01
:1024B0008FEF8BBB80913601882371F20E946E10E2
:1024C000F9CF2FEF3FEF4FE75FE7C701B6010E945B
:1024D000E91A181664F4C111959A8FEF8BBB80919D
:1024E0003801882309F4B8CF0E946E10F8CF20E09D
:1024F00030E0A901C701B6010E949F19D0917B006D
:10250000811106C08FEF8BBBCC23E9F0959A1AC0DE
:1025100020E030E04AE756E4C701B6010E94ED1A18
:1025200020E030E040EC50E40E94A3190E940B1A16
:102530002FEF2BBBC111959A6150704080409040A5
:10254000D9F7C1119598DBBB8CCF809138018823D6
:1025500019F0109238010895809180008330D9F0ED
:102560000E94A50881E080933801E0913D01F0913F
:102570003E0109950E94051080913801882319F0C9
:102580000E946E10F9CF0E943F109598E0913D0196
:10259000F0913E010994089580913801882319F043
:1025A00010923801089580918000833021F10E94BB
:1025B000A50881E080933801E0913D01F0913E0152
:1025C000099580913801882371F080917A0090E01C
:1025D0009BBD8ABD80917800909179000E94241063
:1025E0000E946E10EECF0E943F109598E0913D0141
:1025F000F0913E01099408954F925F926F927F92FD
:102600008F929F92AF92BF92CF92DF92EF92FF9202
:10261000CF9380906E0090906F00A0907000B0906B
:1026200071006091620070916300809164009091EC
:1026300065000E94A80F6B017C0161157105810581
:10264000910521F4C12CD12C7601C394C501B401AC
:102650000E94A80F4B015C01611571058105910570
:1026600021F4812C912C5401839460916A00709123
:102670006B0080916C0090916D000E94A80F2B015F
:102680003C016C157D058E059F0510F42601370170
:1026900080917B00E0E8F2E0C0E89191891718F49E
:1026A000CF5FCF3FD1F76A98809180009FEF980F5E
:1026B000923010F4959A9598833059F58D986A98D0
:1026C00020E030E04AE756E460918100709182009A
:1026D00080918300909184000E94ED1A20E030E008
:1026E00040EC50E40E94A3190E940B1A6115710579
:1026F0008105910539F485990CC06A9BFCCF46C0D1
:102700006A9944C0859BFCCF6150704080409040E6
:10271000D9F7EC2FF0E0E050FE4F222733272C0DA5
:102720003D1DEE1D19F000800BBAF9CF00800BBAE9
:10273000C80CD91CEA1C6E1448F131F45D1430F158
:1027400031F44C1418F116C0000000000000000025
:10275000000000002C0D3D1DEE1D2C0D3D1DEE1D3D
:102760002C0D3D1DEE1D2C0D3D1DEE1D2C0D3D1D9A
:10277000EE1D000049F42C0D3D1DEE1D0000000073
:102780000000F8CF00800BBA6A9BC9CF80917B0014
:102790008BBB0E947C0D80913601882319F00E942A
:1027A0006E10F9CFCF91FF90EF90DF90CF90BF9058
:1027B000AF909F908F907F906F905F904F900C9410
:1027C000730D80913801811130C080912E018130CC
:1027D00031F018F0823041F0089581E001C082E0CC
:1027E00080932E010C94D20A0E94A50881E0809368
:1027F0003801E0913D01F0913E0109950E94730D71
:1028000040E051E063E174E080E092E00E94E61C69
:1028100080913801882319F00E94FC12F9CF0E94A0
:10282000050E10922E010C94C208109238010895E2
:10283000982F907F95BBA89AAA9AEFE9FFE031976D
:10284000F1F700C00000AA98A898EFE9FFE03197DF
:10285000F1F700C00000F0E18F9FC001112485BB9B
:10286000A89AAA9A8FE99FE00197F1F700C00000AB
:10287000AA98A898EFE9FFE03197F1F700C00000AF
:102880000895982F907F95BBAA9AEFE9FFE03197C2
:10289000F1F700C00000AA98EFE9FFE03197F1F7E7
:1028A00000C00000F0E18F9FC001112485BBAA9AEF
:1028B0008FE99FE00197F1F700C00000AA98EFE9C7
:1028C000FFE03197F1F700C00000089581E00C941B
:1028D000411482E00C944114EF92FF921F93CF9326
:1028E000DF931F92CDB7DEB7009771F0182F7C01F0
:1028F0008E2D811B861740F4F70181917F0169833A
:102900000E9418146981F4CF0F90DF91CF911F912D
:10291000FF90EF900895623031F0633031F0613014
:1029200029F4805C03C08C5E01C08C5A80680C94D2
:1029300041141F93CF93DF93EC01862F642F0E94E5
:102940008B1410E0FE01E10FF11D8491882321F02A
:102950000E9418141F5FF6CFDF91CF911F91089549
:10296000EF92FF920F931F93CF93DF938C0188E038
:10297000689FB0011124862F8064E82EC0E0D0E06B
:10298000F801EC0FFD1FF4908C2F8E0D0E94411466
:102990008F2D0E9418142196C830D10589F7DF9138
:1029A000CF911F910F91FF90EF9008951F93CF93B8
:1029B000DF938FE59AEE0197F1F700C0000015BA9A
:1029C00015BA84B3806F84BB84B3876084BB80E313
:1029D00085BBAA9A8FE99FE00197F1F700C000003C
:1029E000AA988FE99FE00197F1F700C0000080E30B
:1029F00085BBAA9A8FE99FE00197F1F700C000001C
:102A0000AA988FE99FE00197F1F700C0000080E2EB
:102A100085BBAA9A8FE99FE00197F1F700C00000FB
:102A2000AA988FE99FE00197F1F700C0000088E2C3
:102A30000E9441148CE00E944114C3E1DBE060E09D
:102A400011E0160FCE010E94B0142896183011F034
:102A5000612FF6CFDF91CF911F910895CF93DF9330
:102A6000D82FC0E0CD1729F08EE10E944114CF5F2E
:102A7000F9CFDF91CF910895CF93DF93D82FC0E0A6
:102A8000CD1729F088E10E944114CF5FF9CFDF9183
:102A9000CF9108958EE00C9441148FE00C94411472
:102AA0008CE00C94411488E00C9441148CE00C945C
:102AB0004114CF93DF93D82FC0E0CD1729F080E1E8
:102AC0000E944114CF5FF9CFDF91CF910895CF934A
:102AD000DF93D82FC0E0CD1729F084E10E94411484
:102AE000CF5FF9CFDF91CF910895CF92DF92EF9230
:102AF000FF920F931F93CF93DF931F92CDB7DEB753
:102B000056E0459F90011124E82FE29FC001E39F0A
:102B1000900D112470E00E94641B8B01CB0166E0D4
:102B200070E00E94501BE82EC12CD12CF12CF41621
:102B3000B9F096012B5F3F4F0217130728F40C15CD
:102B40001D0520F08E2D03C085E001C080E0498383
:102B50000E941814F394F6E0CF0ED11C4981E7CF00
:102B60000F90DF91CF911F910F91FF90EF90DF9029
:102B7000CF9008950E9442100E946E10FDCFA3E1F5
:102B8000B0E0E5ECF5E10C94D71B7C011B016A0178
:102B9000FC0117821682838181FF66C3BE016F5FCD
:102BA0007F4F4B01F7019381F10193FD859193FFD5
:102BB00081911F01882309F453C3853239F493FDB1
:102BC000859193FF81911F01853239F4B70190E01F
:102BD0000E94051D56016501E5CF10E0512C20E053
:102BE0002032A0F48B3269F030F4803259F0833215
:102BF00069F420612CC08D3239F0803339F42160C2
:102C000026C02260246023C0286021C027FD27C081
:102C100030ED380F3A3078F426FF06C0FAE01F9FF7
:102C2000300D1124132F13C06AE0569E300D11246D
:102C3000532E20620CC08E3221F426FD11C3206475
:102C400006C08C3611F4206802C0883641F4F101C8
:102C500093FD859193FF81911F018111C1CF9BEB62
:102C6000980F933018F42061805E06C09BE9980F9E
:102C7000933008F0AAC12F7E26FF16E02F73722E24
:102C8000853621F4F22FF0647F2E08C0863621F4B9
:102C9000622F6068762E02C01111115077FE07C0B6
:102CA0001C3348F444244394410E27E00BC01830F1
:102CB00030F4212F06C027E04CE3442E03C027E068
:102CC00017E0412C560174E0A70EB11CF60160819B
:102CD000718182819381042DA4010E940E1C6C01DC
:102CE000098100FF02C003FF06C071FC07C072FC2F
:102CF00008C0612C08C03DE2632E05C02BE2622EA5
:102D000002C090E2692E802F8C7099F1662011F03C
:102D100084E001C083E0851510F0512C0BC0581AD7
:102D200073FC08C0B70180E290E00E94051D5A9430
:102D3000C9F7F3CF662029F0B701862D90E00E94F5
:102D4000051D03FD03C007E51BE002C003E51BE012
:102D5000F72DF0717F2EF8018491882309F476C253
:102D600071108052B70190E00E94051D0F5F1F4F48
:102D7000F2CF77FE0FC04C0C04FF04C08A81813370
:102D800009F44A94141474F5F8E0F41578F588E021
:102D9000482E2CC076FC2AC0812F90E08C159D0512
:102DA0009CF06CEFC6166FEFD60674F0772D706846
:102DB000772E0AC0E2E0F0E0EC0FFD1FE10FF11DFD
:102DC0008081803319F411501111F4CF77FE0EC0B9
:102DD00044244394410E812F90E0C816D9062CF468
:102DE0001C1904C04424439401C010E077FE07C0BE
:102DF0001C141D043CF496012F5F3F4F05C025E0D5
:102E000030E002C021E030E0662011F02F5F3F4F3C
:102E1000112331F0412F50E04F5F5F4F240F351FDA
:102E2000452D50E02417350714F4521A01C0512CD7
:102E3000872D897049F4552039F0B70180E290E080
:102E40000E94051D5A94F7CF662029F0B701862D00
:102E500090E00E94051D73FC09C0552039F0B701B0
:102E600080E390E00E94051D5A94F7CF77FE5FC083
:102E70009C2D8D2DD7FE02C090E080E0692E782E2B
:102E800040E050E0C601841991099D878C87960126
:102E900026193709280D391D812F90E0EE27FF27CD
:102EA000E81BF90BFF87EE87FFEF6F167F0669F4CB
:102EB000B7018EE290E02B8B3A8B488B598B0E94A6
:102EC000051D598948893A892B89C614D70454F0BD
:102ED0006C857D85661577052CF4F901E40FF51FE7
:102EE000818101C080E371E0671A71084F5F5F4F15
:102EF000EE85FF856E167F066CF0B70190E02B8B98
:102F00003A8B488B598B0E94051D2B893A89488939
:102F10005989CACF6C147D0439F49A81963318F418
:102F2000953311F404FF81E3B70190E04BC08A812F
:102F3000813309F00F7EB70190E00E94051D111149
:102F400005C074FE18C085E490E017C0B7018EE29A
:102F500090E00E94051D82E066246394680EF401EF
:102F6000E80FF11D8081B70190E00E94051D11500E
:102F700041F3862DF1CF85E690E0B7010E94051D53
:102F8000D7FC05C0C114D10439F404FF05C0D194A5
:102F9000C194D1088DE201C08BE2B70190E00E949C
:102FA000051D80E36AE0C616D1042CF08F5FFAE0BD
:102FB000CF1AD108F7CFB70190E00E94051DB701E5
:102FC000C601C0960E94051D41C1833631F083378A
:102FD00079F0833509F058C021C0560172E0A70E80
:102FE000B11CF6018081898301E010E0640114C006
:102FF0005601F2E0AF0EB11CF601C080D18026FF71
:1030000003C0612F70E002C06FEF7FEFC6012B8B12
:103010000E94FA1C8C012B892F7715C05601F2E013
:10302000AF0EB11CF601C080D18026FF03C0612F16
:1030300070E002C06FEF7FEFC6012B8B0E94EF1C88
:103040008C012B892068722E23FD1AC0852D90E0FB
:1030500008171907A8F4B70180E290E00E94051D47
:103060005A94F4CFF60177FC859177FE81916F0138
:10307000B70190E00E94051D51105A9401501109AA
:103080000115110579F7E2C0843611F0893651F542
:10309000560127FF09C0F4E0AF0EB11CF6016081B4
:1030A0007181828193810AC0F2E0AF0EB11CF601FA
:1030B00060817181882777FD8095982F022F0F7688
:1030C00097FF08C090958095709561957F4F8F4FC1
:1030D0009F4F00682AE030E0A4010E944B1DC82EDB
:1030E000C8183EC0022F853721F40F7E2AE030E059
:1030F0001DC0097F8F3691F018F4883559F0B0C0A3
:10310000803719F0883711F0ABC0006104FF09C0A7
:10311000046007C024FF08C0066006C028E030E055
:1031200005C020E130E002C020E132E0560107FF97
:1031300009C0F4E0AF0EB11CF6016081718182819B
:10314000938108C0F2E0AF0EB11CF601608171817D
:1031500080E090E0A4010E944B1DC82EC8180F7794
:1031600006FF0BC0202F2E7FC11650F404FF0AC0AB
:1031700002FD08C0202F2E7E05C0DC2C202F03C0AE
:10318000DC2C01C0D12E24FF0DC0FE01EC0DF11D81
:103190008081803311F4297E09C022FF06C0D394B8
:1031A000D39404C0822F867809F0D39423FD13C0F2
:1031B00020FF06C01C2DD51418F4150D1D19D52C93
:1031C000D51468F4B70180E290E02B8B0E94051DB6
:1031D000D3942B89F5CFD51410F45D1801C0512C70
:1031E00024FF12C0B70180E390E02B8B0E94051DE5
:1031F0002B8922FF17C021FF03C088E590E002C0A1
:1032000088E790E0B7010CC0822F867859F021FD45
:1032100002C080E201C08BE227FD8DE2B70190E0A1
:103220000E94051DC11638F4B70180E390E00E94AA
:10323000051D1150F7CFCA94F401EC0DF11D8081EA
:10324000B70190E00E94051DC110F5CF552009F48B
:10325000C2CCB70180E290E00E94051D5A94F6CFDF
:10326000F7018681978102C08FEF9FEF6396E2E1BD
:103270000C94F31B5058BB27AA270ED070C161D104
:1032800030F066D120F031F49F3F11F41EF456C1A6
:103290000EF4E095E7FB4CC1E92F72D180F3BA1729
:1032A000620773078407950718F071F49EF58AC1C9
:1032B0000EF4E0950B2EBA2FA02D0B01B901900151
:1032C0000C01CA01A0011124FF27591B99F0593F95
:1032D00050F4503E68F11A16F040A22F232F342FDD
:1032E0004427585FF3CF469537952795A795F0402B
:1032F0005395C9F77EF41F16BA0B620B730B840B40
:10330000BAF09150A1F0FF0FBB1F661F771F881FF7
:10331000C2F70EC0BA0F621F731F841F48F487954F
:1033200077956795B795F7959E3F08F0B3CF93953E
:10333000880F08F09927EE0F979587950895D4D0B8
:1033400008F481E008950CD00AC102D140F0F9D010
:1033500030F021F45F3F19F0EBC0511134C1EEC0E1
:103360000FD198F39923C9F35523B1F3951B550B4E
:10337000BB27AA2762177307840738F09F5F5F4F48
:10338000220F331F441FAA1FA9F333D00E2E3AF089
:10339000E0E830D091505040E695001CCAF729D0A3
:1033A000FE2F27D0660F771F881FBB1F26173707F2
:1033B0004807AB07B0E809F0BB0B802DBF01FF2722
:1033C00093585F4F2AF09E3F510568F0B1C0FBC093
:1033D0005F3FECF3983EDCF3869577956795B7955C
:1033E000F7959F5FC9F7880F911D9695879597F977
:1033F0000895E1E0660F771F881FBB1F62177307F0
:103400008407BA0720F0621B730B840BBA0BEE1F04
:1034100088F7E0950895BCD088F09F5790F0B92FB9
:103420009927B751A0F0D1F0660F771F881F991F19
:103430001AF0BA95C9F712C0B13081F0C3D0B1E02B
:103440000895C0C0672F782F8827B85F39F0B93F3B
:10345000CCF3869577956795B395D9F73EF490951B
:103460008095709561957F4F8F4F9F4F0895E89499
:1034700009C097FB3EF490958095709561957F4FBC
:103480008F4F9F4F9923A9F0F92F96E9BB2793956A
:10349000F695879577956795B795F111F8CFFAF47A
:1034A000BB0F11F460FF1BC06F5F7F4F8F4F9F4FAB
:1034B00016C0882311F096E911C0772321F09EE809
:1034C000872F762F05C0662371F096E8862F70E06F
:1034D00060E02AF09A95660F771F881FDAF7880F49
:1034E0009695879597F90895990F0008550FAA0B9F
:1034F000E0E8FEEF16161706E807F907C0F0121607
:103500001306E407F50798F0621B730B840B950B09
:1035100039F40A2661F0232B242B252B21F408955E
:103520000A2609F4A140A6958FEF811D811D0895FB
:1035300097F99F6780E870E060E008959FEF80EC66
:10354000089500240A941616170618060906089509
:1035500000240A9412161306140605060895092E6F
:103560000394000C11F4882352F0BB0F40F4BF2BDE
:1035700011F460FF04C06F5F7F4F8F4F9F4F08951E
:1035800057FD9058440F551F59F05F3F71F0479514
:10359000880F97FB991F61F09F3F79F087950895F9
:1035A000121613061406551FF2CF4695F1DF08C018
:1035B000161617061806991FF1CF86957105610535
:1035C00008940895E894BB2766277727CB0197F9DD
:1035D00008958ADF08F48FEF08950BD0C0CFB1DFD4
:1035E00028F0B6DF18F0952309F0A2CFA7CF112459
:1035F000EACFC6DFA0F3959FD1F3950F50E0551F9A
:10360000629FF001729FBB27F00DB11D639FAA2737
:10361000F00DB11DAA1F649F6627B00DA11D661F86
:10362000829F2227B00DA11D621F739FB00DA11DA7
:10363000621F839FA00D611D221F749F3327A00D61
:10364000611D231F849F600D211D822F762F6A2FFD
:1036500011249F5750408AF0E1F088234AF0EE0F82
:10366000FF1FBB1F661F771F881F91505040A9F78F
:103670009E3F510570F05CCFA6CF5F3FECF3983EC4
:10368000DCF3869577956795B795F795E7959F5FF6
:10369000C1F7FE2B880F911D9695879597F9089590
:1036A000AA1BBB1B51E107C0AA1FBB1FA617B70768
:1036B00010F0A61BB70B881F991F5A95A9F7809584
:1036C0009095BC01CD01089597FB072E16F4009448
:1036D00007D077FD09D00E94501B07FC05D03EF4AF
:1036E000909581959F4F0895709561957F4F0895AE
:1036F000689401C0E8948F929F92CF93DF930E94C9
:10370000861BDF91CF919F908F90089588249924F4
:10371000F401E401B0E49F93AA279A158B049C045A
:10372000ED05FE05CF05D007A10798F4AD2FDC2FDE
:10373000CF2FFE2FE92D982C892E982F872F762FAB
:10374000652F542F432F322F2227B85031F7BF91C6
:1037500027C01B2EBF91BB27220F331F441F551FAD
:10376000661F771F881F991F881C991CEE1FFF1F5B
:10377000CC1FDD1FAA1FBB1F8A149B04EC05FD058F
:10378000CE05DF05A007B10748F08A189B08EC09B1
:10379000FD09CE09DF09A00BB10B21601A94E1F6F7
:1037A0002EF49401AF01BE01CD01000C08952F92BB
:1037B0003F924F925F926F927F928F929F92AF92C1
:1037C000BF92CF92DF92EF92FF920F931F93CF930E
:1037D000DF93CDB7DEB7CA1BDB0B0FB6F894DEBFA5
:1037E0000FBECDBF09942A88398848885F846E84CB
:1037F0007D848C849B84AA84B984C884DF80EE8015
:10380000FD800C811B81AA81B981CE0FD11D0FB61D
:10381000F894DEBF0FBECDBFED010895283008F04B
:1038200027E03327DA01990F311D87FD916000965B
:103830006105710539F432602E5F3D9330E32A95BE
:10384000E1F708959F3F30F080387105610509F078
:103850003C5F3C5F3D93913008F08068911DDF93A1
:10386000CF931F930F93FF92EF92192F987F969506
:10387000E92F96959695E90FFF27EB54F44F99277A
:103880003327EE24FF24A701E7010590089407944D
:1038900028F4360FE71EF81E491F511D660F771FCB
:1038A000881F991F0694A1F70590079428F4E70E46
:1038B000F81E491F561FC11D770F881F991F661FCD
:1038C0000694A1F70590079428F4F80E491F561F97
:1038D000C71FD11D880F991F661F771F0694A1F778
:1038E0000590079420F4490F561FC71FD81F990F42
:1038F000661F771F881F0694A9F78491109517708B
:1039000041F0D695C79557954795F794E7941A9542
:10391000C1F7EBE5FBE06894159015913591659141
:10392000959105907FE27395E118F10A430B560BD0
:10393000C90BD009C0F7E10CF11E431F561FC91F68
:10394000D01D7EF4703311F48A95E6CFE8940150CF
:1039500030F0080F0AF40027021708F4202F2395EF
:10396000022F7A3328F079E37D932A95E9F710C086
:103970007D932A9589F606949795679537951795BF
:103980001794E118F10A430B560BC90BD00998F0B4
:1039900023957E9173957A3308F070E37C9320131E
:1039A000B8F77E9170617D9330F0839571E37D93DC
:1039B00070E32A95E1F71124EF90FF900F911F918A
:1039C000CF91DF91992787FD90950895FB01DC0148
:1039D00002C005900D9241505040D8F70895FC0167
:1039E0000590615070400110D8F7809590958E0F2A
:1039F0009F1F0895FC016150704001900110D8F79D
:103A0000809590958E0F9F1F08950F931F93CF93CE
:103A1000DF93182F092FEB018B8181FD03C08FEFFE
:103A20009FEF20C082FF10C04E815F812C813D81BD
:103A3000421753077CF4E881F9819F012F5F3F4FC4
:103A400039832883108306C0E885F985812F09957D
:103A5000892B29F72E813F812F5F3F4F3F832E8394
:103A6000812F902FDF91CF911F910F910895A0E0AA
:103A7000B0E0EDE3FDE10C94E71BFE0135966191AA
:103A80007191AF0180914F01909150010E94BF153B
:103A9000E2E00C94031CFA01AA27283051F12031EE
:103AA00081F1E8946F936E7F6E5F7F4F8F4F9F4FD2
:103AB000AF4FB1E03ED0B4E03CD0670F781F891F14
:103AC0009A1FA11D680F791F8A1F911DA11D6A0FE2
:103AD000711D811D911DA11D20D009F468943F9195
:103AE0002AE0269F11243019305D3193DEF6CF0194
:103AF0000895462F4770405D4193B3E00FD0C9F75A
:103B0000F6CF462F4F70405D4A3318F0495D31FDC6
:103B10004052419302D0A9F7EACFB4E0A695979519
:103B2000879577956795BA95C9F7009761057105EF
:103B300008959B01AC010A2E069457954795379539
:103B40002795BA95C9F7620F731F841F951FA01D93
:103B50000895DC01CB01FC01E199FECF06C0FFBB5B
:103B6000EEBBE09A31960DB20D9241505040B8F73D
:103B70000895E199FECF9FBB8EBBE09A99278DB344
:103B80000895DC01A40FB51F4150504048F0CB010F
:103B9000840F951F2E910E94D21D41505040D0F7A6
:103BA0000895262FE199FECF9FBB8EBBE09A019727
:103BB0000DB2021631F02DBB0FB6F894E29AE19ADD
:103BC0000FBE0895262FE199FECF9FBB8EBB2DBB64
:103BD0000FB6F894E29AE19A0FBE01960895F89410
:023BE000FFCF15
:103BE200FF0000007A440000803F00409C46CDCC9C
:103BF200CC3D010000C8420024F47F800000803FD9
:103C0200000000000000000002000000005A07004F
:103C12000000002531302E3366487A004578616312
:103C220074202020202020004D696E2E206A6974A5
:103C320074657200253375004F66662020202020AF
:103C42000053696E676C652020004D756C74697055
:103C52006C650054726967676572200025382E33DF
:103C6200666D73004F66662020202020202000759C
:103C72006E74696C2072656C20006D696E20202064
:103C82002020202000756E74696C2073746F7000A0
:103C920025382E366600202535754D487A002535A3
:0E3CA2002E316625250025382E3266487A0020
:00000001FF
